:1000000010308A00952D0000FF00030E8301A1002F
:100010000A08A0008A010408A2007708A300780853
:10002000A4007908A5007A08A6007B08A70083131E
:1000300083120B1E1D288B1836288C308400801EDE
:1000400023288C1A3928220884002308F700240862
:10005000F8002508F9002608FA002708FB00200808
:100060008A00210E8300FF0E7F0E09008A110A16F6
:10007000BD2A8A110A16522C0A108A100A11820708
:10008000123401341034013400340034003410349C
:10009000C7340534133401340134003401340234DC
:1000A000033401340934023422340034013401347D
:1000B0000034A034323409340434003400340134C0
:1000C000033401340234003409342134103401344F
:1000D000003401342234323400340734053482349D
:1000E000033410340034FF3404340334093404344A
:1000F0001E340334523400346F340034623400341C
:1001000065340034723400347434003420340034E4
:100110004D340034653400346534003472340034B6
:100120006D340034613400346E34003414340334DC
:100130004D34003465340034653400347234003496
:100140004D3400346F34003475340034733400346B
:10015000653400341E3403344C34003469340034C4
:100160006D34003469340034743400346534003440
:100170006434003445340034643400346934003469
:1001800074340034693400346F3400346E34003415
:10019000343422340534013409340234A1340134B6
:1001A00009340134A13400340534093419340134DC
:1001B00029340334153400342534013495340334A0
:1001C0007534013481340234953401347534053486
:1001D0008134013405340134093430340934313484
:1001E0001534813425347F34753408349534023421
:1001F00081340634C034C0340A148A100A118207CC
:100200000D340A34203447344234413420344334EA
:100210006F346E34743472346F346C346C346534CF
:100220007234203465346E34613462346C34653435
:100230006434213420340D340A3400340A148A1012
:100240000A1182074534723472346F3472342034A8
:1002500069346E3420344434313432345F345734AA
:100260007234693474346534283429342C3420349D
:1002700075346E346B346E346F3477346E342034AE
:1002800074347934703465343A342034303478340A
:100290002534783421340D340A3400340A148A1099
:1002A0000A11820745347834703465346334743409
:1002B00069346E34673420346F346E3465342034DE
:1002C0006F3466343A340D340A340934203430340F
:1002D0007834253478340D340A34093430347834A1
:1002E000253478340D340A3400340A148A100A1183
:1002F00082070D340A340D340A3425346434203432
:1003000000340A148A100A1182075F3453344134CE
:100310004534203400340A148A100A1182075F34ED
:10032000533445344534203400340A148A100A11F9
:1003300082075F3453344D34203400340A148A1059
:100340000A11820753345234453451342034003476
:100350000A148A100A118207433452344534513446
:10036000203400340A148A100A11820745345234AA
:1003700045345134203400340A148A100A1182079B
:100380003F345234453451343D34253478342034AC
:1003900000340A148A100A11820747346534743411
:1003A0005F3453347434613475347334203400341E
:1003B0000A148A100A11820743346C34653461349C
:1003C00072345F3446346534613474347534723455
:1003D0006534203400340A148A100A118207533419
:1003E000653474345F346634653461347434753420
:1003F00072346534203400340A108A140A118207DA
:100400005334653474345F34413464346434723446
:10041000653473347334203400340A108A140A119A
:1004200082074734653474345F344434653473343C
:10043000633472346934703474346F3472342034F9
:1004400000340A108A140A11820753346534743454
:100450005F344434653473346334723469347034D3
:1004600074346F347234203400340A108A140A1140
:1004700082074734653474345F3443346F346E34E8
:100480006634693467347534723461347434693471
:100490006F346E34203400340A108A140A11820733
:1004A0005334653474345F3443346F346E3466349B
:1004B00069346734753472346134743469346F3438
:1004C0006E34203400340A108A140A11820747342B
:1004D000653474345F3449346E3474346534723442
:1004E0006634613463346534203400340A108A146D
:1004F0000A1182075334653474345F3449346E34DE
:100500007434653472346634613463346534203451
:1005100000340A108A140A118207533479346E3475
:10052000633468345F344634723461346D34653416
:10053000203400340A108A140A1182073F345334DD
:100540005234453451343D34253478342034003429
:100550000A108A140A1182075334743461347434D3
:10056000653449346E3463346F346D3470346134BF
:100570007434613462346C3465342834253478340E
:100580002C34253478342934203400340A108A1469
:100590000A1182072A344334443428342534783409
:1005A0002934203400340A108A140A1182072A34AC
:1005B00052344434283425347834293420340034F7
:1005C0000A108A140A1182074C346F343D342534E2
:1005D000783420344C346C343D3425347834203431
:1005E00000340A108A140A1182073F34443452340A
:1005F0003D3425347834203400340A148A140A1126
:10060000820721344C3454343D342534783420343A
:1006100000340A148A140A1182073F344C345434CB
:100620003D3425347834203400340A148A140A11F5
:1006300082074434493452343D3400340A148A1455
:100640000A118207213453346534743443343D3401
:1006500025347834203400340A148A140A118207AD
:100660003F3443345234453451343D3425347834A6
:10067000203400340A148A140A1182074434613485
:10068000743461344C3465346E343D3425347834FC
:10069000203400340B088316D70083128B132912E1
:1006A000290883168700831207120830F80000001B
:1006B00000000000F8176D2BF8138316D60C831278
:1006C00003180716031C071278176D2B7813F80B05
:1006D0005D2B00000000000007160A308400840B28
:1006E0006F2B00000000F81B5C2B781B662B831619
:1006F000D71F7D2B83128B1783168312003483162A
:10070000D51B942B0F30F700540EF7050A307702F3
:1007100003188D2B3030F7078F2B5508F707770814
:10072000D60083124A2383160F30D4050A305402B0
:1007300003189C2B30309E2BD5135508D407540832
:10074000D60083124A23003483164F08F700F708B7
:1007500083120319B02B013077020319B02BDD2B64
:1007600000308316880086108312861483164F0B80
:10077000BE2B061383120617C12B83160613831292
:100780000613831650088312880008308316D100A0
:100790005108D103003A031DC82B0611831206111C
:1007A000831606118312061583164F0BDB2B0613D7
:1007B0008312061383164B2C83122B08073C031C51
:1007C000E22B2A142B08073C031C0B2C8316D201A6
:1007D000520883121E218316D20AF700D600831214
:1007E0004A23263083165202031DE82B4F08D400FB
:1007F0005730D50083127F2321308316D600831211
:100800004A230D308316D60083124A230A308316FA
:10081000D60083124A232B08073C031C102C2A14F1
:100820002B08073C031C4A2C8316D2015208831262
:100830004E218316D20AF700D60083124A231730BE
:1008400083165202031D162C0130D4005730D500F8
:1008500083127F2319308316D300530883124E214D
:100860008316D30AF700D60083124A231E3083165C
:100870005302031D2D2CD4015730D50083127F2342
:100880000D308316D60083124A230A308316D60011
:1008900083124A23831683120034FF3083168800A4
:1008A000CF014E084F020318662C86108312861063
:1008B00083164D084F0784008312080880008316B2
:1008C0008610831286148316CF0A512C83120034AB
:1008D000B101B001B201AF01AC01AE01AD01AB0895
:1008E000031D732C2A14AB08031D832CFD017D0806
:1008F0008121FD0AF7008316D60083124A230530B2
:100900007D02031D772C01308316CF00D030D0003C
:100910008312A4238316CF018030D0008312A42336
:10092000AB08031D942C2A14AB08031DA42CFD0155
:100930007D088B21FD0AF7008316D60083124A2317
:1009400005307D02031D982C01308316CF00D8306E
:10095000D0008312A4238316CF010130D00083126C
:10096000A423AB08031DB52C2A14AB08031DC52C0A
:10097000FD017D089521FD0AF7008316D60083123C
:100980004A2304307D02031DB92C01308316CF00A9
:10099000F330D0008312A4238316CF011630D00089
:1009A0008312A4238316CF010B30D0008312A4231B
:1009B00000342B08073C031CDE2C2A142B08073CB0
:1009C000031CEC2C53308316D60083124A235F306D
:1009D0008316D60083124A2383164D08F700F708C2
:1009E00083120319082D013077020319212D0230DB
:1009F000770203193A2D033077020319532D04307F
:100A0000770203196C2D053077020319852D9E2D71
:100A10002B08073C031C0D2D2A142B08073C031C34
:100A2000202D43308316D60083124A234F3083167D
:100A3000D60083124A2320308316D60083124A231D
:100A4000C32D2B08073C031C262D2A142B08073C1A
:100A5000031C392D43308316D60083124A234930B4
:100A60008316D60083124A2320308316D6008312C1
:100A70004A23C32D2B08073C031C3F2D2A142B08A7
:100A8000073C031C522D45308316D60083124A239F
:100A90004F308316D60083124A2320308316D600A7
:100AA00083124A23C32D2B08073C031C582D2A14FC
:100AB0002B08073C031C6B2D45308316D600831290
:100AC0004A2349308316D60083124A2320308316E6
:100AD000D60083124A23C32D2B08073C031C712D1B
:100AE0002A142B08073C031C842D4D308316D60096
:100AF00083124A234F308316D60083124A232030B4
:100B00008316D60083124A23C32D2B08073C031CEF
:100B10008A2D2A142B08073C031C9D2D4D3083166B
:100B2000D60083124A2349308316D60083124A2303
:100B300020308316D60083124A23C32D2B08073C8E
:100B4000031CA32D2A142B08073C031CC22D3F3085
:100B50008316D60083124A2328308316D6008312C8
:100B60004A2383164D08D4005730D50083127F23C3
:100B700029308316D60083124A2320308316D600EC
:100B800083124A23C32D403083164D07CE00013017
:100B9000CF004E08D0008312A4238316CF0101306A
:100BA000D0008312A42300342B08043C031CD92D4D
:100BB0002A142B08043C031CEE2D8316C0014008A8
:100BC000831215238316C00AF700D60083124A2326
:100BD000043083164002031DDF2D831283163F0865
:100BE0008400801F092E83122B08043C031CF92D5E
:100BF0002A142B08043C031C072E49308316D60008
:100C000083124A2320308316D60083124A231D2ED6
:100C1000831683122B08043C031C0F2E2A142B0866
:100C2000043C031C1D2E4F308316D60083124A232A
:100C300020308316D60083124A232B08043C031C61
:100C4000222E2A142B08043C031C352E5430831604
:100C5000D60083124A234F308316D60083124A23CC
:100C60003D308316D60083124A2383163F08840042
:100C700000081F39F700F708831203194C2E0130C2
:100C800077020319602E023077020319742E0330A5
:100C900077020319882E9C2E2B08043C031C512E2E
:100CA0002A142B08043C031C5F2E44308316D60004
:100CB00083124A2320308316D60083124A23AF2E94
:100CC0002B08043C031C652E2A142B08043C031C2F
:100CD000732E49308316D60083124A2320308316A0
:100CE000D60083124A23AF2E2B08043C031C792E16
:100CF0002A142B08043C031C872E45308316D6008B
:100D000083124A2320308316D60083124A23AF2E43
:100D10002B08043C031C8D2E2A142B08043C031CB6
:100D20009B2E3F308316D60083124A232030831631
:100D3000D60083124A23AF2E2B08073C031CA12E9A
:100D40002A142B08073C031CAA2E07308316D60052
:100D500083124A238316CD018312D924AF2E2B0888
:100D6000043C031CB42E2A142B08043C031CE32E61
:100D7000023083163F078400840A0008C100840300
:100D80000008C0007730D60083124A2356308316FD
:100D9000D60083124A233D308316D60083124A239D
:100DA00083164108D4005730D50083127F23831661
:100DB0004008D4005730D50083127F23203083169B
:100DC000D60083124A232B08043C031CE82E2A1465
:100DD0002B08043C031C172F043083163F078400A4
:100DE000840A0008C10084030008C0007730D600E0
:100DF00083124A2349308316D60083124A233D309A
:100E00008316D60083124A2383164108D400573034
:100E1000D50083127F2383164008D4005730D500B5
:100E200083127F2320308316D60083124A232B0897
:100E3000043C031C1C2F2A142B08043C031C4B2FBE
:100E4000063083163F078400840A0008C10084032B
:100E50000008C0007730D60083124A234C30831636
:100E6000D60083124A233D308316D60083124A23CC
:100E700083164108D4005730D50083127F23831690
:100E80004008D4005730D50083127F2320308316CA
:100E9000D60083124A23003401308316CF004D0858
:100EA000D0008312A42301308316CF00F030D0008D
:100EB0008312A4238316CF01D0018312A4238316A7
:100EC000CF01D0018312A42301308316CF00FA3062
:100ED000D0008312A423AA142B08033C031C712FF7
:100EE0002A142B08033C031C7F2F5A308316D6008C
:100EF00083124A2320308316D60083124A230034FB
:100F000001308316CD0083124C2701308316CF00A9
:100F1000D030D0008312A42302308316410784000E
:100F2000840A0008C30084030008C2008038C4009B
:100F30004308C500CF014408D0008312A423023027
:100F4000831641078400840A0008C3008403000854
:100F5000C20080388312B2000130B100AA142B08FD
:100F6000033C031CB42F2A142B08033C031CC72F7B
:100F700041308316D60083124A2353308316D6009D
:100F800083124A2320308316D60083124A2300346A
:100F90000B088316C80083128B13291229088316A5
:100FA0008700831207120830F800000000000000DC
:100FB000F817EB2FF8138316C70C831203180716C4
:100FC000031C07127817EB2F7813F80BDB2F0000A8
:100FD0000000000007160A308400840BED2F00008B
:100FE0000000F81BDA2F781BE42F8316C81FFB2F95
:0A0FF00083128B178316831200345E
:1010000001308316CF004130D0008A118312A4230F
:101010008A15C9308316CD000130CE008A118312A3
:101020004D248A152B08013C031C17282A142B0871
:10103000013C031C40284C308316D6008A118312D1
:101040004A238A1554308316D6008A1183124A2304
:101050008A153D308316D6008A1183124A238A15D9
:1010600083164908D4005730D5008A1183127F2394
:101070008A1520308316D6008A1183124A238A15D6
:10108000AD08031D4628AE08031933292B08053C7B
:10109000031C4B282A142B08053C031C64284430ED
:1010A0008316D6008A1183124A238A15523083167A
:1010B000D6008A1183124A238A1520308316D6005F
:1010C0008A1183124A238A15AE08031D6B282D0846
:1010D000103C03186D28103070282E08FA002D08D7
:1010E0008316CB004B0883122C078316CC00831287
:1010F000AB08031D7C282A14AB08031DA228831605
:10110000CD014D088A1183123A238A158316CD0A20
:10111000F700D6008A1183124A238A1508308316F5
:101120004D02031D81284B08D4005730D5008A1189
:1011300083127F238A1520308316D6008A118312EA
:101140004A238A1501308316CF00D0008A118312FA
:10115000A4238A1501308316CF00F030D0008A1105
:101160008312A4238A158316CF01D0018A1183121A
:10117000A4238A158316CF014B08D0008A1183124D
:10118000A4238A1583164C0883122C020318F62810
:10119000AB08031DCC282A14AB08031DE3282C0838
:1011A0008A113C208A158316CD00D4005730D50013
:1011B0008A1183127F238A1520308316D6008A1164
:1011C00083124A238A152C088A113C208A1583161B
:1011D000CD00CF014D08D0008A118312A4238A15B7
:1011E0002D080319AE03AD03AC0AC22801308316E3
:1011F000CF00FA30D0008A118312A4238A15AD08DB
:10120000031D1129AE08031D112983164B080F3940
:10121000003A031D12290130CD008A1183124C2798
:101220008A1583168312AA142B08023C031C192961
:101230002A142B08023C031C322944308316D600A2
:101240008A1183124A238A1553308316D6008A11D5
:1012500083124A238A1520308316D6008A118312FE
:101260004A238A153E29AA1C3729AA103E29013093
:101270008316CD008A118312D9248A1500340630D2
:10128000831641078400840A0008FA0084030008DA
:10129000C2007A08C3008312AE01AD01AB08031D82
:1012A00052292A14AB08031D8D29023083164107E9
:1012B0008400840A0008CA0084030008C9004A08A0
:1012C000CB00CC014730D6008A1183124A238A15FD
:1012D00044308316D6008A1183124A238A15283097
:1012E0008316D6008A1183124A238A1583164B0867
:1012F000D4005730D5008A1183127F238A152930F4
:101300008316D6008A1183124A238A152030831649
:10131000D6008A1183124A238A158316C601C80192
:101320004608BA3C031C2E2B46088A1183123C2027
:101330008A15F8008316C5017808C40001304607F5
:101340008A1183123C208A15F8008316C700831285
:10135000AB08031DAC292A14AB08031DFB29693017
:101360008316D6008A1183124A238A153D308316CC
:10137000D6008A1183124A238A1583164608D400A0
:101380005730D5008A1183127F238A15283083169F
:10139000D6008A1183124A238A1583164408D40082
:1013A0005730D5008A1183127F238A152C3083167B
:1013B000D6008A1183124A238A1520308316D6005C
:1013C0008A1183124A238A1583164708D40057309E
:1013D000D5008A1183127F238A1529308316D600FF
:1013E0008A1183124A238A1520308316D6008A1167
:1013F00083124A238A150230831641078400840A27
:101400000008CA0084030008C9004A08FA0147021C
:10141000031D2B2BFA08031D2B2B4708F700023066
:101420007702831203191D2A0330770203196C2AED
:10143000223077020319882AC32A0230831646070E
:101440008A1183123C208A15F8008316C50178089A
:10145000C400033046078A1183123C208A15F80025
:101460008316CB017808CA00FA000030C4047A0859
:10147000C5048312AB08031D3E2A2A14AB08031DC2
:101480006B2A8316C90149088A118312C6228A155C
:101490008316C90AF700D6008A1183124A238A15D7
:1014A000043083164902031D432A4408D4005730F0
:1014B000D5008A1183127F238A1529308316D6001E
:1014C0008A1183124A238A1520308316D6008A1186
:1014D00083124A238A15C32A0230831641078400E7
:1014E000840A0008CA0084030008C9000F39CB0031
:1014F0004A080039CC0048084B02031D822ACC0858
:101500000319862AC80A4408C60790298312C32AE9
:1015100002308316C607C4020030031C0130C50226
:101520008312AB08031D952A2A14AB08031DC22A97
:101530008316C90149088A118312D3228A1583169A
:10154000C90AF700D6008A1183124A238A1504308B
:1015500083164902031D9A2A4408D4005730D50047
:101560008A1183127F238A1529308316D6008A11A7
:1015700083124A238A1520308316D6008A118312DB
:101580004A238A15C32A831645084302031CD22A1C
:10159000031DCE2A420844020318D22A4508C3007C
:1015A0004408C20046088312AC0083164308831225
:1015B000AE00831642088312AD00AB08031DE12A7A
:1015C0002A14AB08031D282B4C308316D6008A1131
:1015D00083124A238A156F308316D6008A1183122C
:1015E0004A238A153D308316D6008A1183124A2376
:1015F0008A152C088316D4005730D5008A1183121F
:101600007F238A1505308316C90049088A11831281
:10161000E0228A158316C90AF700D6008A118312C0
:101620004A238A15093083164902031D052B8312AC
:101630002D088316D4005730D5008A1183127F23DA
:101640008A1520308316D6008A1183124A238A1500
:1016500083162E2B2D2B4408C60790298312AD0824
:10166000031D8B2BAE08031D8B2B2B08073C031C83
:101670003A2B2A142B08073C031C452B07308316F2
:10168000D6008A1183124A238A152B08073C031CB3
:101690004A2B2A142B08073C031C7D2B023083168F
:1016A00041078400840A0008CA0084030008C900B6
:1016B0004A08CB00CC01CD014D088A118312F122DA
:1016C0008A158316CD0AF700D6008A1183124A23A1
:1016D0008A15043083164D02031D5C2B4B08D40081
:1016E0005730D5008A1183127F238A152030831644
:1016F000D6008A1183124A238A158316CD018A11D6
:101700008312D9248A1501308316CD008A118312E1
:10171000D9248A158C2B002000342B08013C031C93
:10172000922B2A142B08013C031C062C340884003D
:1017300000088316C30001308312340784000008B8
:101740008316C40002308312340784008316C50157
:101750000018C50A02308312340784008316C601BC
:101760008018C60A7830C7008A118312C8278A15E4
:1017700083164308D4005730D5008A1183127F2383
:101780008A1520308316C7008A118312C8278A154C
:1017900079308316C7008A118312C8278A158316E9
:1017A0004408D4005730D5008A1183127F238A154C
:1017B00020308316C7008A118312C8278A1561302A
:1017C0008316C7008A118312C8278A158316450815
:1017D000D4005730D5008A1183127F238A15203018
:1017E0008316C7008A118312C8278A1562308316B0
:1017F000C7008A118312C8278A1583164608D400A9
:101800005730D5008A1183127F238A150130831641
:10181000CF004530D0008A118312A4238A150130ED
:101820008316CF000530D0008A118312A4238A15B5
:1018300001308316CF00F030D0008A118312A42328
:101840008A158316CF01D0018A118312A4238A1529
:101850008316CF010330D0008A118312A4238A1586
:101860008316CF01D0018A118312A4238A1534086C
:10187000840000088316C300CF014308D0008A11FA
:101880008312A4238A1501303407840000088316CC
:10189000C300CF014308D0008A118312A4238A1504
:1018A00001308316CF00FA30D0008A118312A423AE
:1018B0008A15003483164214023041078400840ADA
:1018C0000008C40084030008C3000F39F70044086F
:1018D0000039FA007A08031D732C01307702831255
:1018E0000319742C83167B2C0230B1000130B00038
:1018F0008D23BA2C831683122B08073C031C812CE2
:101900002A142B08073C031CB62C0230831641070F
:101910008400840A0008C40084030008C3000F394F
:10192000C50044080039C600C70147088A11831260
:101930001E238A158316C70AF700D6008A11831260
:101940004A238A15063083164702031D952C450845
:10195000D4005730D5008A1183127F238A15203096
:101960008316D6008A1183124A238A1583164210E1
:101970008312BA2C8316421CC52C0130CD008A116B
:1019800083124C278A15CB2C83160130CD008A1187
:101990008312D9248A1500348316401401303F077E
:1019A00084000008F700F70883120319002D0130A6
:1019B000770203192C2D033077020319582D0530B7
:1019C00077020319842D063077020319B32D0730EF
:1019D00077020319E52D0830770203190F2E09301D
:1019E00077020319392E0A3077020319682E0B305B
:1019F000770203198F2E0C3077020319B62EDD2ED5
:101A00002B08043C031C052D2A142B08043C031C42
:101A10001E2D8316C10141088A118312C9218A151E
:101A20008316C10AF700D6008A1183124A238A1549
:101A30000A3083164102031D0B2D83123108023C2C
:101A40000319272D310B282DB208031D282D2B2D0E
:101A5000831640108312222F2B08043C031C312DC7
:101A60002A142B08043C031C4A2D8316C10141088B
:101A70008A118312D8218A158316C10AF700D6006D
:101A80008A1183124A238A150E3083164102031DE0
:101A9000372D83123108023C0319532D310B542D7D
:101AA000B208031D542D572D831640108312222F88
:101AB0002B08043C031C5D2D2A142B08043C031C3A
:101AC000762D8316C10141088A118312EB218A15F4
:101AD0008316C10AF700D6008A1183124A238A1599
:101AE0000C3083164102031D632D83123108023C22
:101AF00003197F2D310B802DB208031D802D832DFE
:101B0000831640108312222F2B08043C031C892DBE
:101B10002A142B08043C031CA22D8316C101410882
:101B20008A118312FC218A158316C10AF700D60098
:101B30008A1183124A238A150C3083164102031D31
:101B40008F2D8312B1080319A72D310BAF2D8316EA
:101B50003F08C1008A11831280278A15B22D83168F
:101B600040108312222F2B08043C031CB82D2A148A
:101B70002B08043C031CD12D8316C10141088A1196
:101B800083120D228A158316C10AF700D6008A1126
:101B900083124A238A150F3083164102031DBE2D7E
:101BA0008312B1080319DB2D310BD72DDB2D310842
:101BB000023C031DE12D83163F08C10083123F2123
:101BC000E42D831640108312222F2B08043C031CA3
:101BD000EA2D2A142B08043C031C032E8316C10192
:101BE00041088A11831221228A158316C10AF7003F
:101BF000D6008A1183124A238A150F3083164102B8
:101C0000031DF02D8312310B062E0A2E3108023CE3
:101C1000031D0B2E0E2E831640108312222F2B082D
:101C2000043C031C142E2A142B08043C031C2D2EE8
:101C30008316C10141088A11831235228A15831641
:101C4000C10AF700D6008A1183124A238A1512307E
:101C500083164102031D1A2E8312310B302E342EAF
:101C60003108023C031D352E382E83164010831296
:101C7000222F2B08043C031C3E2E2A142B08043C64
:101C8000031C572E8316C10141088A1183124C226E
:101C90008A158316C10AF700D6008A1183124A23D7
:101CA0008A15123083164102031D442E8312310B14
:101CB0005A2E5E2E3108023C031D642E83163F0807
:101CC000C10083125A24672E831640108312222FDC
:101CD0002B08043C031C6D2E2A142B08043C031C07
:101CE000862E8316C10141088A11831263228A1548
:101CF0008316C10AF700D6008A1183124A238A1577
:101D00000E3083164102031D732E83123108023CEC
:101D1000031D8B2E8E2E831640108312222F2B082C
:101D2000043C031C942E2A142B08043C031CAD2EE7
:101D30008316C10141088A11831276228A158316FF
:101D4000C10AF700D6008A1183124A238A150E3081
:101D500083164102031D9A2E83123108023C031D93
:101D6000B22EB52E831640108312222F2B08043C6E
:101D7000031CBB2E2A142B08043C031CD42E8316F0
:101D8000C10141088A11831289228A158316C10A6A
:101D9000F700D6008A1183124A238A150C30831665
:101DA0004102031DC12E83123108023C031DD92EAE
:101DB000DC2E831640108312222F831640108312CC
:101DC0002B08073C031CE52E2A142B08073C031C98
:101DD000F02E07308316D6008A1183124A238A1503
:101DE0002B08073C031CF52E2A142B08073C031C68
:101DF000212F013083163F0784000008C100C20173
:101E000042088A1183129A228A158316C20AF700A1
:101E1000D6008A1183124A238A150630831642029D
:101E2000031D002F4108D4005730D5008A118312BA
:101E30007F238A1520308316D6008A1183124A2305
:101E40008A15222F0030831640180130003A031DF6
:101E5000762F83122B08073C031C2F2F2A142B08E4
:101E6000073C031C6F2F8316C10141088A1183129E
:101E7000A8228A158316C10AF700D6008A11831298
:101E80004A238A15123083164102031D352F83120F
:101E900031088316D4005730D5008A1183127F236E
:101EA0008A152C308316D6008A1183124A238A158C
:101EB00032088316D4005730D5008A1183127F234D
:101EC0008A1529308316D6008A1183124A238A156F
:101ED00020308316D6008A1183124A238A1583166E
:101EE000CD018A118312D9248A15831683120034F6
:101EF0008316401401303F0784000008F7000A30C1
:101F000077028312031DA02F33088316C10002300D
:101F10003F078400840A0008C30084030008C2004D
:101F20004308FA01C4007A08C50041088400440847
:101F300080000130CD008A1183124C278A15E52FCD
:101F40008316401083122B08073C031CA82F2A1469
:101F50002B08073C031CB32F07308316D6008A11C9
:101F600083124A238A152B08073C031CB82F2A1416
:101F70002B08073C031CE42F013083163F07840025
:101F80000008C100C20142088A1183122C238A155D
:101F90008316C20AF700D6008A1183124A238A15D3
:101FA000063083164202031DC32F4108D400573068
:101FB000D5008A1183127F238A1520308316D6001C
:101FC0008A1183124A238A15E52F003083164018A0
:101FD0000130003A031DF22FCD018A118312D9245A
:101FE0008A158316831200340A168A11442C0A12A9
:0A1FF0008A1578088A110A165A2C87
:102000002B08073C031C05282A142B08073C031C3B
:102010002C288316C10141080A128312FD220A16D8
:102020008316C10AF700D6000A1283124A230A1641
:10203000043083164102031D0B284008D40057309A
:10204000D5000A1283127F230A1620308316D60089
:102050000A1283124A230A1683164008F700023038
:102060007702831203196528043077020319662862
:1020700006307702031967280830770203196828A9
:102080000A307702031969280C30770203196A288D
:102090000E30770203196B281030770203196C2871
:1020A0001230770203196D281430770203196E2855
:1020B0001630770203196F281A3077020319702837
:1020C0001E307702031971287228AF28AF28AF2875
:1020D000AF28AF28AF28AF28AF28AF28AF28AF2848
:1020E000AF28AF282B08073C031C77282A142B089D
:1020F000073C031C822807308316D6000A1283127D
:102100004A230A162B08073C031C87282A142B088D
:10211000073C031CAE288316C10141080A12831232
:1021200009230A168316C10AF700D6000A12831281
:102130004A230A16043083164102031D8D284008E5
:10214000D4005730D5000A1283127F230A1620309C
:102150008316D6000A1283124A230A16AF280034C7
:1021600001308316CF004030D0000A128312A4231E
:102170000A16AB308316CD000130CE000A1283124E
:102180004D240A162B08033C031CC7282A142B08CD
:10219000033C031CF0284C308316D6000A1283122D
:1021A0004A230A1654308316D6000A1283124A2391
:1021B0000A163D308316D6000A1283124A230A16E5
:1021C00083162B08D4005730D5000A1283127F23C0
:1021D0000A1620308316D6000A1283124A230A16E2
:1021E0008316AB1FF3282B1CAF2AAB1EAE2A01307F
:1021F000CF00D0010A128312A4230A16AD30831631
:10220000CD000130CE000A1283124D240A162B088D
:10221000023C031C0C292A142B08023C031C352900
:1022200053308316D6000A1283124A230A16453009
:102230008316D6000A1283124A230A163D308316EB
:10224000D6000A1283124A230A1683162D08D400D8
:102250005730D5000A1283127F230A1620308316C6
:10226000D6000A1283124A230A1601308316CF00C1
:10227000F030D0000A128312A4230A16AD30831660
:10228000CD001030CE000A1283124D240A162B08FE
:10229000023C031C4C292A142B08023C031C752900
:1022A00044308316D6000A1283124A230A164C3091
:1022B0008316D6000A1283124A230A163D3083166B
:1022C000D6000A1283124A230A1683162E08D40057
:1022D0005730D5000A1283127F230A162030831646
:1022E000D6000A1283124A230A1601308316CF0041
:1022F000F130D0000A128312A4230A16013083168B
:10230000CF00F230D0000A128312A4230A16013043
:102310008316CF00D0000A128312A4230A160130BC
:102320008316CF00F130D0000A128312A4230A16BC
:1023300001308316CF00F230D0000A128312A4239A
:102340000A1683162E08083C031DA82A0230BE0078
:102350003E08093C031CCB298312AB08031DB1299D
:102360002A14AB08031DC829AD3083163E0784002C
:102370000008BF00D4005730D5000A1283127F2313
:102380000A1620308316D6000A1283124A230A1630
:102390008316BE0AA829AF30BD003D08BF000A124F
:1023A0008312D4250A1683163D088400000860397C
:1023B000F700F70EF70C0730F705770883120319BB
:1023C000EA29013077020319122A02307702031931
:1023D0003A2A592A2B08043C031CEF292A142B08FB
:1023E000043C031C082A8316BF013F080A1283120B
:1023F0009E210A168316BF0AF700D6000A1283121E
:102400004A230A16053083163F02031DF52983125D
:1024100083163D08BF000A128A158312CC240A16BF
:102420008A11A62A2B08043C031C172A2A142B08FD
:10243000043C031C302A8316BF013F080A12831292
:10244000A8210A168316BF0AF700D6000A128312C3
:102450004A230A16053083163F02031D1D2A8312E4
:1024600083163D08BF000A128A15831278270A16C0
:102470008A11A62A2B08043C031C3F2A2A142B0885
:10248000043C031C582A8316BF013F080A1283121A
:10249000B2210A168316BF0AF700D6000A12831269
:1024A0004A230A16053083163F02031D452A83126C
:1024B000A62A2B08073C031C5E2A2A142B08073C7B
:1024C000031C692A07308316D6000A1283124A2396
:1024D0000A162B08073C031C6E2A2A142B08073CFB
:1024E000031C9F2A83163D08840000086039F7000A
:1024F000770EC100C10C0730C105C20142080A12A3
:102500008312BC210A168316C20AF700D6000A12EB
:1025100083124A230A16053083164202031D7E2ABF
:102520004108D4005730D5000A1283127F230A16BF
:1025300020308316D6000A1283124A230A16831605
:10254000CD010A128312D9240A16A62AAD2A8316AF
:10255000CD010A128312D9240A168316BB2A2B082E
:102560001E39003A0319BB2A2B081E39BF00C000D0
:1025700083120020831683120034831606148312FC
:102580000618402C00302A180130013C031DDA2ABD
:1025900000302A180130FD000D308316D6000A12D3
:1025A00083124A230A160A308316D6000A128312AF
:1025B0004A230A162A1001308316CF00F430D000C7
:1025C0000A128312A4230A1674308316CD00023037
:1025D000CE000A1283124D240A167408F6007508FC
:1025E000FC00AB08031DF52A2A14AB08031D2D2B94
:1025F00049308316D6000A1283124A230A16523033
:102600008316D6000A1283124A230A163D30831617
:10261000D6000A1283124A230A1676088316D400BB
:102620005730D5000A1283127F230A162C308316E6
:10263000D6000A1283124A230A167C088316D40095
:102640005730D5000A1283127F230A1620308316D2
:10265000D6000A1283124A230A16761F512B2B0822
:10266000073C031C342B2A142B08073C031C4D2B5E
:1026700042308316D6000A1283124A230A165230B9
:102680008316D6000A1283124A230A1620308316B4
:10269000D6000A1283124A230A160A1268240A165E
:1026A000DA2BF61F722B2B08013C031C582B2A1423
:1026B0002B08013C031C712B53308316D6000A12E1
:1026C00083124A230A1643308316D6000A12831255
:1026D0004A230A1620308316D6000A1283124A2390
:1026E0000A16DA2B761C942B2B08033C031C792B3F
:1026F0002A142B08033C031C922B43308316D6006C
:102700000A1283124A230A164F308316D6000A1281
:1027100083124A230A1620308316D6000A12831227
:102720004A230A16B020DA2BF61CBA2B2B08033CDE
:10273000031C9B2B2A142B08033C031CB42B433093
:102740008316D6000A1283124A230A1649308316CA
:10275000D6000A1283124A230A1620308316D600A6
:102760000A1283124A230A160A128A1500200A1630
:102770008A11DA2B761DDA2B2B08033C031CC12BA4
:102780002A142B08033C031CDA2B31308316D600A5
:102790000A1283124A230A164F308316D6000A12F1
:1027A00083124A230A1620308316D6000A12831297
:1027B0004A230A16F61DFB2B2B08033C031CE12BB6
:1027C0002A142B08033C031CFA2B31308316D60045
:1027D0000A1283124A230A1649308316D6000A12B7
:1027E00083124A230A1620308316D6000A12831257
:1027F0004A230A163F2C761E1C2C2B08033C031C74
:10280000022C2A142B08033C031C1B2C3230831689
:10281000D6000A1283124A230A164F308316D600B6
:102820000A1283124A230A1620308316D6000A128F
:1028300083124A230A163F2CF61E3F2CAB08031DB9
:10284000222C2A14AB08031D3A2C32308316D600F2
:102850000A1283124A230A1649308316D6000A1236
:1028600083124A230A1620308316D6000A128312D6
:102870004A230A160A128A158D230A168A11BD2ABE
:102880008B108A110A1223288C1E442C1808B500BC
:102890001A08F800B51C4E2C1812181600008A15DC
:1028A0000A12F72F831686138030831286060A12C7
:1028B0008A15F42F0A168A117808F7005E3077021D
:1028C00003197B2C763077020319802C3C30770279
:1028D0000319852C3E3077020319892C4130770289
:1028E00003198D2C423077020319922C5330770252
:1028F0000319972CA72C0130340784008003A72CE0
:10290000013034078400800AA72C34088400800337
:10291000A72C34088400800AA72C023034078400D6
:102920000014A72C0230340784008014A72C34082C
:1029300084008001013034078400800102303407B4
:10294000840000100230340784008010A72C8C1201
:102950008A110A1223283A08F80139020318B32C05
:102960003908F700BF2CF7010830BB00B90DF70D8F
:102970003A0877020318F700F80DBB0BB62C0034A9
:102980003708F700B71BC82C381DDD2C2030CD2CA4
:10299000F709F70A7708B7002D30F800A8018B1B5C
:1029A000A8178B1378088316D6000A1283124A23BD
:1029B0000A16A81B8B17381DB8153708B9006430E4
:1029C000BA00AB247708B70078083030031DEF2C2D
:1029D0003818FF2CB819FF2C381A2030F12CB811F8
:1029E0003812F807A8018B1BA8178B1378088316D9
:1029F000D6000A1283124A230A16A81B8B1737081F
:102A0000B9000A30BA00AB247708B7007808303034
:102A1000031D0E2DB8191C2D381A2030F807A801F7
:102A20008B1BA8178B1378088316D6000A12831203
:102A30004A230A16A81B8B173030B707A8018B1B37
:102A4000A8178B1337088316D6000A1283124A235D
:102A50000A16A81B8B178A110A167E2D8316861359
:102A60008312861301308316860000308800FF3001
:102A7000831288008316861083128614831606112B
:102A80008312061583160613831206138316061285
:102A9000831206120B138B138B1B4B2D8316011302
:102AA00083120B168B10C0308B0405080739AB005E
:102AB0002B08073C031C5D2D2A142B08073C031C24
:102AC0008B2DB60136080A1275210A16B60AF700D0
:102AD000A8018B1BA8178B1377088316D6000A1240
:102AE00083124A230A16A81B8B1704303602031DD3
:102AF000622D2B08B7001830B800C02CA8018B1B22
:102B0000A8178B1320308316D6000A1283124A238B
:102B10000A16A81B8B178A110A16C32D0C1E8E2DA0
:102B2000370899008A110A16FF2D84011F3083058A
:102B3000063083169F008312291229088316870006
:102B400083120716193083169900263098009030AA
:102B5000831298002912290883168700831207160A
:102B6000193083169900263098009030831298000F
:102B7000291229088316870083120716FF30A9003F
:102B8000B5012A102E2D340884008001013034074D
:102B900084008001023034078400001002303407C2
:102BA000840080108316061400308312061801304A
:102BB000003A031DE22DA8018B1BA8178B138B1461
:102BC000A81B8B17851DF62D34088400013080006A
:102BD0003407840001308000023034078400001084
:102BE0000230340784008010F42D072EB601360819
:102BF0000A12FC200A16B60AF700B7008E2D1D3007
:102C00003602031DF72D83168C16052E83126300E2
:02400E00F13F80
:00000001FF
